:020000040000FA
:100000004828000000000000A8000308A9001030E4
:100010008506A003031D1428A1030F3021052730F6
:1000200003192830A00026140B111F302405031DCE
:100030003C2819302506031D3C2810302006031DDE
:100040003C28271C252827103C28FF302C050319A5
:100050003C2800302406031935283C30AA00230828
:10006000AA022C082A0203183C28AC03A71C3B2830
:10007000A00A27143C28A0032908830028080900A7
:100080000000000000000000000000000000000070
:1000900083160313803081002830850000308600ED
:1000A000831207309F00A0308B0007308500FF309F
:1000B00086003230A5002830A0000E30A2000F309C
:1000C000A3000430AB000030A400A600A70081000C
:1000D000261C7028B220CB20A61C7028A610342124
:1000E0000630051A103E8500FF302406261D7A28AA
:1000F000FE309C208600AD20FF308600A320053016
:00000001FF
